:10000000A00E0020D11700001940000025180000A4
:100010002518000025180000251800000000000029
:10002000000000000000000000000000F9150000C2
:100030002518000000000000A5150000F93F000091
:100040009117000091170000911700009117000010
:100050009117000091170000911700009117000000
:1000600091170000911700009117000091170000F0
:1000700091170000911700009117000091170000E0
:1000800091170000911700009117000091170000D0
:1000900091170000911700009117000091170000C0
:1000A00091170000911700009117000091170000B0
:1000B00091170000911700009117000091170000A0
:1000C0009117000091170000911700009117000090
:1000D0009117000091170000911700009117000080
:1000E0009117000091170000911700009117000070
:1000F0009117000091170000911700009117000060
:1001000053B94AB9002908BF00281CBF4FF0FF317E
:100110004FF0FF3000F074B9ADF1080C6DE904CE7A
:1001200000F006F8DDF804E0DDE9022304B07047D2
:100130002DE9F047089E0D4604468846002B4DD118
:100140008A42944668D9B2FA82F252B101FA02F3B5
:10015000C2F1200120FA01F10CFA02FC41EA030885
:1001600094404FEA1C45210CB8FBF5FE1FFA8CF7B2
:1001700005FB1E8341EA03430EFB07F199420BD9AD
:100180001CEB03030EF1FF3080F01E81994240F218
:100190001B81AEF1020E63445B1AA4B2B3FBF5F00F
:1001A00005FB103344EA034400FB07F7A7420AD9D2
:1001B0001CEB040400F1FF3380F00881A74240F2F9
:1001C000058164440238E41B40EA0E4000211EB160
:1001D000D4400023C6E90043BDE8F0878B4208D92C
:1001E000002E00F0EE800021C6E900050846BDE8BB
:1001F000F087B3FA83F100294AD1AB4202D382429D
:1002000000F2F980841A65EB030301209846002E62
:10021000E2D0C6E90048DFE702B9FFDEB2FA82F2B7
:10022000002A40F09180A1EB0C054FEA1C471FFA11
:100230008CFE0121B5FBF7F307FB1350250C45EAB3
:1002400000450EFB03F0A84208D91CEB050503F19D
:10025000FF3802D2A84200F2CB8043462D1AA4B246
:10026000B5FBF7F007FB105544EA05440EFB00FE12
:10027000A64508D91CEB040400F1FF3502D2A645BF
:1002800000F2BB802846A4EB0E0440EA03409EE740
:10029000C1F120078B4022FA07FC4CEA030C20FA3C
:1002A00007F405FA01F31C43FD404FEA1C4900FA2C
:1002B00001F3B5FBF9F8200C1FFA8CFE09FB185569
:1002C00040EA054508FB0EF0A84202FA01F20BD9FC
:1002D0001CEB050508F1FF3A80F08880A84240F247
:1002E0008580A8F1020865442D1AA4B2B5FBF9F087
:1002F00009FB105544EA054500FB0EFEAE4508D942
:100300001CEB050500F1FF346CD2AE456AD902380A
:10031000654440EA0840A0FB0294A5EB0E05A54207
:10032000C846A64656D353D05EB1B3EB080265EB80
:100330000E0505FA07F722FA01F3CD401F43C6E97F
:1003400000750021BDE8F087C2F1200320FA03F117
:100350000CFA02FC25FA03F395400D434FEA1C47C3
:100360001FFA8CFEB3FBF7F107FB11302B0C43EAAD
:10037000004301FB0EF0984204FA02F408D91CEB8A
:10038000030301F1FF382FD298422DD9023963447B
:100390001B1AADB2B3FBF7F007FB103345EA034578
:1003A00000FB0EF3AB4208D91CEB050500F1FF384A
:1003B00016D2AB4214D902386544ED1A40EA014125
:1003C00038E73146304607E78646E5E61846FAE65E
:1003D0004B45A9D2B9EB020864EB0C0E0138A3E738
:1003E0004046EAE7204694E74146D1E7D0467BE71E
:1003F000023B654432E7084609E76444023842E7B5
:10040000704700BF0B6801330B60014B1B68184736
:1004100000000020014B1860704700BF0000002062
:1004200007B50B46002102460191034801A900F0DF
:10043000E5F803B05DF804FB050400002DE9F84F72
:10044000B0F8189019F00808044693460DD0012919
:100450000CBF49F0100949F02009A0F818908BF35F
:100460001188BFF36F8FBDE8F88F09F007090229E3
:1004700007D1204603F017FC0028F0D00128238B79
:100480004ED16769218B002F15DA256821F007010D
:10049000C4E9008841F0010121830026218B01F08D
:1004A000070ACA4502D0A368002B5AD10DB9002E05
:1004B00071D0002356E001F007035A1F012A1ED80D
:1004C00021F00701062B256889B2C4E900880AD10A
:1004D0003DB1638B2A46126801339BB2002AFAD1E0
:1004E000638341F002012183204603F0DCFB0646D2
:1004F0000028D3D0238B43F020032383CDE7042BA4
:100500000CD121F0070189B22183204603F0CBFBF7
:1005100005460028C1D041F0200121830025BCE719
:10052000032809D1226923F00703166843F0060364
:10053000238300252F46B1E7042806D1226923F042
:100540000703566843F00403F2E7052806D1226941
:1005500023F00703966843F00503E9E700252E46DC
:10056000E8E7012341F0080121838BF31188BFF3F1
:100570006F8FFBB985BB16B11F492046B0474FF0BE
:100580002003EFF3118B83F31188BFF36F8F238B5D
:1005900023F008032383238BDA0625D523F01003E9
:1005A00023830121B4F8189009F0070900297FF48A
:1005B0005EAF54E7A1680029DCD0D1F80090D1F8F3
:1005C00004B03B4652462046D847B9F1000FD1D07F
:1005D0004946D9F80090F2E729463B465246204664
:1005E0002D6803F07CFBC5E713F020011EBF23F04C
:1005F000200323830221D5E70B3D00002DE9F04FB6
:1006000091B08B46029092461C4600259AF8000055
:1006100008B928465FE325280AF1010707D0029BA5
:10062000594698470028C0F25683013512E2182235
:1006300000210AA803F01EFD9AF80130252B78D07E
:1006400000221046964694461646394617F8013B56
:100650002B2B00F09D8000F29480202B00F09B80DB
:10066000232B00F09B802EB19DF8306046F00406ED
:100670008DF83060BCF1000F05D09DF8306046F079
:1006800008068DF83060BEF1000F05D09DF830608F
:1006900046F010068DF8306028B19DF8300040F02B
:1006A00020008DF830002AB19DF8302042F0400241
:1006B0008DF830209DF8302002F04400442803D10A
:1006C0006FF386128DF830209DF830202A2B42F0EF
:1006D00080028DF830207BD19DF8312042F001025C
:1006E0004B1C8DF831201A782E2A9DF831200CBF32
:1006F0000121002161F341028DF8312074D15A7833
:100700002A2A6AD0013300210A26184610F8012B44
:10071000A2F13007092F40F28E809DF830200E9113
:10072000C2F3400040EAD17161F341028DF83020FC
:100730005AE00AF102078DF833309DF83130D907BD
:1007400040F1498154F8049BB9F1000F07DA9DF894
:10075000302042F004028DF83020C9F100095A0718
:1007600040F1428154F8048BB8F1000F80F24181CE
:100770009DF831306FF341038DF831304FF0FF3881
:1007800037E12D2B0CD0302B7FF46DAF01225CE7CD
:100790004FF0010C59E74FF0010E56E7012054E7E6
:1007A000012652E70CFB0202303A33461E4616F889
:1007B000010BA0F13007092FF4D9994293D09DF88D
:1007C00030100D92D20F62F341018DF830108AE79C
:1007D0000B4600224FF00A0CE8E79DF8312042F06A
:1007E00004028DF8312002331F4617F8012B6C2AC2
:1007F00041D025D8682A2BD06A2A46D04C2A4CD022
:100800001F4617F8012B9DF831308DF83320782AD8
:1008100000F2D980572A4DD8412A03D0453A022AFE
:1008200000F2D1809DF83230042262F302038DF889
:10083000323001239EE006FB01213039034664E794
:10084000742A26D07A2ADBD19DF8313006220DE0B9
:100850005A78682A9DF8312006D1012161F3C60239
:100860008DF831209F1CCCE71346022262F3C603A9
:100870008DF83130C5E75A786C2A9DF8312001D1C6
:100880000421EBE713460322F0E79DF831300522FF
:10089000ECE79DF831300722E8E7BDF8303023F46B
:1008A000F04323F0020343F4804343F00203ADF826
:1008B0003030A6E7A2F15801202900F2848001A07F
:1008C00050F821F089090000C7090000C70900009D
:1008D000C7090000C7090000C7090000C7090000D8
:1008E000C7090000C709000025080000C70900006B
:1008F00089090000490900002508000025080000BA
:1009000025080000C709000049090000C7090000C8
:10091000C7090000C7090000C709000091090000CD
:1009200089090000AD090000C7090000C7090000DF
:10093000AD090000C709000089090000C7090000CF
:10094000C7090000890900009DF83210012003F05A
:10095000780360F30201402B8DF8321002BF9DF83E
:10096000301041F001018DF83010632A31D1003B85
:1009700018BF01239DF83020C2F340010B4363F3FD
:1009800041028DF83020D8E69DF832100220DEE7D3
:100990009DF8322003F07803A3F14000032161F3B6
:1009A000020243428DF832204341E3E79DF83220B2
:1009B000032113F0780F61F302028DF8322014BF87
:1009C00001230023D6E79DF8303043F001038DF872
:1009D00030300023CEE79DF93020002AB4BFDDF887
:1009E00034904FF0FF39BAE69B077FF5C7AEDDF8CC
:1009F00038809DF831100023CDE90D339DF8323059
:100A000003F00703012BC1F3C30138D1CB1E042B24
:100A100022D8DFE803F003090921210054F8043B40
:100A2000DA17CDE90A3206E0073424F00704F4E8C7
:100A30000223CDE90A239DF8303013F0030656D087
:100A400002983B465246594603F028FA0028C0F265
:100A500042810544BA46D9E554F8043B01294FEADE
:100A6000E372CDE90A3205D19DF828300A930023BC
:100A70000B93E0E70229DED1BDF92830D0E7022B45
:100A800023D1CB1E042B13D8DFE803F0030A0A128C
:100A9000120022680A920023201D0B930446CAE725
:100AA000E01D20F00700F0E80223CDE90A23F5E776
:100AB00054F8043B0A9301294FF000030B93D3D061
:100AC0000229B8D1BDF82830D0E7042B09D1E31DA5
:100AD00023F0070303F10804D3E90023CDE90A2337
:100AE000A9E7032B04BF54F8043B0A93A3E79DF83E
:100AF00033007828AED8622822D825283FF48FAD5D
:100B00005828A7D10DF126030093DDE90A0104ABB3
:100B10000CAA03F07DF98246B8F1000F0DF1260012
:100B20000CDB9DF83020A0EB0A036FF3861298458A
:100B30008DF8302002D9A8EB03030D9380463DE0E9
:100B40006338152886D801A252F820F0CD0B00009A
:100B5000310C0000550A0000550A0000550A00003B
:100B6000550A0000310C0000550A0000550A00002B
:100B7000550A0000550A00008B0C0000590C0000BB
:100B80005D0C0000550A0000550A0000A50B00008E
:100B9000550A0000590C0000550A0000550A0000D3
:100BA000590C0000B8F1000FDDF828A00ADB41461F
:100BB000504603F03FFA0AEB00080026BAF1000F96
:100BC0000CD147E7504603F02EFAF4E70A9B8DF864
:100BD000103000260DF1100A0DF11108A8EB0A03E0
:100BE00006B101339DF83220D00668D50233520693
:100BF0000D9948BF0E9A0B4448BF9B18B9F1000FDE
:100C000076DD9DF83020A9EB0309C2F3800303933E
:100C100053076DD4500661D546B1029B5946304604
:100C20009847002857DB039B01351E46302356E0CA
:100C30001E070FD413F0100618BF2026DDE90A2383
:100C4000002BBFF65FAF524263EB4303CDE90A23AB
:100C50002D2657E72B26F1E7002653E70A9840B3E5
:100C60000DF1260300930CAA04AB002103F0D0F889
:100C7000BDF8323003F0EF0343F4F04343F01003C8
:100C80008246ADF83230002646E70A9B07293FF638
:100C9000E1AEDFE801F00C04060C08080C0C1D7036
:100CA000D8E61D80D6E6EA17C3E90052D2E61D60F9
:100CB000D0E6DFF8C8A006460AF105088EE711075E
:100CC00048BF013393E7184603935946029B984760
:100CD0000028039B04DA11B0BDE8F08F20234D44B7
:100CE0004A46002AA5EB090109F1FF39EBDC0D4664
:100CF00036B1029B5946304698470028EBDB013558
:100D00009DF83230D90601D41A0706D5029B594600
:100D1000302098470028DEDB01359DF83230DB06B5
:100D200007D59DF83300029B594698470028D2DB2F
:100D300001350D9E2E44731B002B16DC0298434692
:100D40005246594603F0AAF80028C4DB0544A944DA
:100D5000A9EB0503002B7FF77DAE029B59462020AF
:100D600098470028B7DB0135F2E7029B594630204F
:100D700098470028AFDB0135DDE700BFE04A0000FF
:100D800008B504464FF02002EFF3118382F3118877
:100D9000BFF36F8F03F032F9204600F083FF034862
:100DA00002F074FF00F0BCFCFCE700BFE64A000064
:100DB000F8B505464FF02003EFF3118683F3118851
:100DC000BFF36F8F094B1C685CB1094FD4E9013246
:100DD000002D08BF13460BB1387898472468002CC3
:100DE000F4D186F31188BFF36F8FF8BD080200209D
:100DF000100200201FB50F4B1A68BAB901221A6001
:100E00000D4A07CA01AB83E807000C4A4AB193E8D0
:100E1000070003F04EF9002005B05DF804EBFFF782
:100E2000C7BF82F31188BFF36F8FF4E705B05DF899
:100E300004FB00BF0400002010020020B3400000AB
:100E4000F0B589B06E4601460546304603F03DF8E0
:100E500096E80700174C84E807002078274638B347
:100E6000154B002119606B1C0DD0144816464FF429
:100E7000004C134A0023E6FB0C01FFF741F9012166
:100E8000281A03F0BFFB02F0A9F80120FFF790FF3A
:100E900097E8070005AB83E807000A4A1AB193E810
:100EA000070003F0F3F8FFF7A5FF02F04FF92078F1
:100EB00009B0F0BD10020020040000203F420F00E6
:100EC00040420F008D40000010B50748074C01F06C
:100ED00061FD074B1860204600F0C6FE2046FFF774
:100EE00099FA002010BD00BF0F4B0000F50E000066
:100EF0001C0200200A2838B5074D044604D1286892
:100F000083680D215B68984728688368E1B25B6855
:100F10009847204638BD00BF1C020020084B70B522
:100F2000C31A0D4607499B10044659430648402200
:100F300002F0ECFF2B4601462046BDE87040184702
:100F400034020020B76DDBB6B446000073B50C4C1C
:100F50000C4A4023041B00930D460B460A49A4107B
:100F600061430646094802F0FDFF011E05DA3046DE
:100F70002B4602B0BDE87040184702B070BD00BFFC
:100F800034020020D53F0000B76DDBB6B446000048
:100F9000002270B501210446104600F05BFB0020E2
:100FA00000F03AFB0F4801F0C9FB0F4B984215D1F6
:100FB00003F0A4F926690D49304602F0C3FE00286B
:100FC0000BDB246909490125356404F11C0002F09A
:100FD000B9FE002801DBE564002070BD6FF004005D
:100FE000FBE700BF251000000000AD0B0C4900001E
:100FF00001460C2309484B4370B5C418D4E90E567A
:1010000000224033A263184402F06DFF2DB1324636
:101010002B460348BDE87040184770BD34020020DD
:10102000B446000010B1012804D07047034B1B6C7C
:101030005B0701D1FFF7DCBF704700BF340200201F
:1010400008B54FF02003EFF3118183F31188BFF34C
:101050006F8F124A136843F0020013F0010310600F
:101060000CD04FF08042D2F80C34D2F80C2413F09C
:10107000010303D00A4802F036FF012381F31188EF
:10108000BFF36F8F23B1BDE808400020FFF7B0BF6A
:10109000BDE80840012003F03BB900BF84020020F6
:1010A000740200201FB500220123CDE90223094A62
:1010B000CDF800D06B46CDF804D002F084FF0028B4
:1010C00005DB4FF480420023684601F007FF05B0BE
:1010D0005DF804FBF33F0000094BBFF35B8F53E85F
:1010E000002F22F0020143E800100028F7D1BFF3DF
:1010F0005B8FD30702D4012001F030BB704700BFE3
:10110000840200202DE9F0413949BFF35B8F074687
:10111000012251E8003F41E800200028F9D1BFF347
:101120005B8F33B9334934484B60CB608A6002F03F
:101130001CFE7B1E012B2FD8012F07D14FF08043BF
:10114000D3F81C3403F00303012B25D003F076F908
:10115000044618B9294B1B78002B41D14FF02003CE
:10116000EFF3118683F31188BFF36F8F0124DFF84B
:1011700090804FF08045D5F81834D5F81824D20364
:101180000CD503F00303012B01D0012F06D10CB3C2
:1011900086F31188BFF36F8FBDE8F081ACB13046A4
:1011A00000F0CCFAD5F81835002BE4D1D5F804219D
:1011B000002AE0D0C5F80431D5F804310123C5F880
:1011C0001835C8F88031AB60D5E70021212002F046
:1011D00083F9E7E74FF080430222C3F80423DBE7FB
:1011E0004FF080430222C3F808230646BFE700BF42
:1011F000880200202402002050020020D208002093
:1012000000E100E0044A1368C81A20F07F4003445C
:10121000136002F0B3BA00BF9C0200202DE9F8432E
:10122000860006F1804600F1500406F58836A400D9
:10123000A4B204F180444FF48037D6F84035DFF88B
:101240006C8021F07F4504F588348740D8F80495F8
:10125000A3EB090323F07F4329F07F42012BC6F85B
:10126000402502D1132003F0EBF909F10202AB1A79
:1012700023F07F43B3F5000F88BF1546002323609A
:101280002368C8F8447325F07F43C6F84035D8F882
:101290000435994506D0EB1A023B23F07F43B3F5A2
:1012A000000F01D8BDE8F8832B46CFE700100140BE
:1012B00070B5154D154C00262B68002006B170BD89
:1012C000D4F80423D203FAD5D4F84021002AF6D06A
:1012D000C4F84061D4F840214FF48032C4F8482368
:1012E000D4F84015D4F80465721A22F07F42B2F5A2
:1012F000000F88BF314601261BB16A6828609847F5
:10130000DAE72B60DBE700BF90020020001001400D
:1013100038B50F4C00254FF48033C4F80855C4F895
:1013200004330C4B4FF40032C3F8802101212A46CC
:10133000112000F08FF9112000F06EF90123064A08
:10134000A360022023601360FFF7DCFE284638BD4F
:101350000010014000E100E098020020134AB0F1C3
:10136000FF3F14BF03461346013B002B1CDD934295
:10137000A8BF13460E4AD2F804050E4A1168401A57
:1013800010F4000F20F07F4218BF002301321344F5
:10139000094A0A48106000205060044A934294BFF2
:1013A000C9188918FFF73ABF0023E3E7FFFF7F0062
:1013B000001001409C020020900200200512000055
:1013C000044BD3F80405044B1B68C01A20F07F407F
:1013D000704700BF001001409C020020014802F04D
:1013E0009BBA00BF1849000010B5044618B90D4B50
:1013F0000D485B689847616808290DD031F00403F7
:101400000AD011F0020108D00848214602F0EDFF91
:10141000002323600023636010BD2068142202F0C3
:1014200029FEF7E74C000020264B0000A002002018
:1014300008B508B34368042B10D101220368BFF339
:101440005B8F53E8001F002903D143E800200028E8
:10145000F7D1BFF35B8F0BD1002008BD53B10068FB
:101460004FF0FF324FF0FF3301F05EFC0028F3D065
:101470000348F2E70348F0E76FF4E040EDE700BF10
:10148000E98FFFFFEA8FFFFF08B5D0B14368042B57
:1014900011D100220368BFF35B8F53E8001F0129BD
:1014A00003D143E800200028F7D1BFF35B8F074842
:1014B00008BF104608BD3BB1006801F0ADFC00203C
:1014C000F8E76FF4E040F5E70148F3E7E98FFFFF45
:1014D000EA8FFFFF10B5044618B9164B16485B6833
:1014E00098476368042B23D0082B21D0CBB92368FD
:1014F000BBB912484FF0FF324FF0FF33214601F0E5
:1015000041FB08B923681BB90A4B0D485B68984733
:1015100020681422002102F0ADFD636843F002034D
:101520006360206802F09FFF636843F0010363601B
:1015300010BD00BF4C000020264B0000A002002080
:101540004C4B000008B5064906484023142202F01F
:1015500031FFBDE808400449044802F03FBA00BF2B
:10156000BC020020A00200203049000020490000F9
:10157000094A0A49936809689967094958674B6895
:1015800043F080534B60002383F31188BFF36F8FC8
:101590009368986F704700BF78080020544A000095
:1015A00000ED00E012498A684FF030001044EFF37C
:1015B000098C80E8F01F202080F31188BFF36F8F23
:1015C0000C4F4FF000664A6A8A603E60506F0023FD
:1015D000536780F3118804B5104600F08BFABDE81C
:1015E000044002F1300090E8F01F8CF30988704746
:1015F0007808002004ED00E01EF0040F0CBFEFF3AC
:101600000880EFF30980816911F8021C0229FFD0DC
:1016100001B502F0FDFC01BD43B2002B08DB012245
:1016200000F01F0002FA00F05B09024A42F82300B2
:10163000704700BF00E100E0054B420900F01F00C9
:1016400053F82220012303FA00F01040704700BF36
:1016500000E100E043B2002BA8BF03F1604301F1B9
:101660000101B8BF064B4FEA4111ACBF03F561431E
:1016700000F00F00C9B2B4BF195483F800137047CB
:1016800014ED00E042F8203C009B42F81C3C0A4963
:10169000019B42F8183C029B42F8143C21F00101E6
:1016A0004FF0807342F8043C42F8081C0023203AB3
:1016B00002654367704700BFFD3D0000094A0346CD
:1016C000906870B113F1160F406E05D0A0F12002A2
:1016D0009A4205D8834203D2814228BF0020704736
:1016E000002070477808002008B5094B98600D4627
:1016F000144600F0FFF9204685F30988002163B6FF
:1017000081F31188BFF36F8F0022002302F076FB74
:1017100078080020014910220A60704710ED00E0AF
:1017200072B6404080F31188BFF36F8FBFF34F8FC5
:1017300030BF62B6BFF36F8F704700BF72B64940CB
:1017400081F3118820BF80F3118862B6704700BF13
:1017500030BFFFF7FDBF00BF0B4A08B50B4B22F0AF
:101760007F029A60BFF34F8FBFF36F8FD3F888204B
:1017700022F47002C3F8882001F036F901F01EFF50
:1017800000F08EF901F054F90000000000ED00E0D7
:1017900001B572B60B4A106A00281EBF0021116203
:1017A00002F052FE62B6EFF30580A0F110004FEA9E
:1017B000C0000549014409C99847BDE801400349F3
:1017C00008470000780800202C470000FD190000A1
:1017D000002080F31488BFF36F8F02F035FF0020E4
:1017E0000D490860BFF34F8F0C4880F3088800F064
:1017F00025F9202080F3118809484FF40261401830
:1018000080F30988EFF314800221084380F31488E1
:10181000BFF36F8FFFF7A0FF94ED00E0A00E002054
:1018200020100020EFF30880EFF3098101B5724624
:1018300000F056F801BD00BF38B5194B14469A6A3E
:101840009A6A9A6A0546900719D5586B9A6A1206E1
:1018500015D519B19A6A22F080029A629A6A9A6A38
:101860009A6AD1060ED49B6A9A070BD400200C4AC0
:10187000936A43F0FF0393620023237038BD6FF037
:101880001500EBE7064B5B681B05EFD52946FFF714
:1018900015FF0028EAD080F309880220E7E700BF9F
:1018A00000ED00E00D4B9A6A9A6A9A6A920508D593
:1018B0009A6B9A6A120404D518B19A6A22F400420B
:1018C0009A62064B9A6A9A6AD20558BF9A6A9A6ACD
:1018D000002042F47F429A620870704700ED00E0F9
:1018E00070B5414B5B688AB00E46C3F30803002510
:1018F00085F31188BFF36F8F02F07F41B1F17F4F05
:1019000011D102F00C0108290DD0110701D40646AF
:1019100001250022033B8DF80720032B5DD8DFE86B
:1019200003F004474B4F2E46F3E72F4BDC6A14F0CD
:10193000020452D1DA6A520022D593F828203AB133
:101940000DF1070201213046FFF776FF044617E04C
:1019500093F829202AB10DF107010120FFF7A2FF1A
:10196000F4E75A8D92B25AB19A6A9A6A9A6A9A6A56
:101970009A6A9A6A9A6A6FEA02426FEA12429A6215
:101980009DF8073093B92022314602A802F067FB88
:10199000099B25B3C3F3080222B96FEA53236FEA08
:1019A0004323099302A9204602F030FB0AB070BD20
:1019B0000DF107020021C6E70DF107010020CDE778
:1019C000094B9A6A9A6A9A6A9A6A9A6A9A6A9A6AA7
:1019D0006FEA02426FEA12429A620024D0E723F4CF
:1019E000FF7323F00103DCE700ED00E0024A5369D6
:1019F00043F010035361704700ED00E0044B996819
:101A0000586A884203D003494FF080520A607047F9
:101A10007808002004ED00E00749D1F89020002369
:101A2000C2F307221846934200D17047C1F898309C
:101A3000C1F8A0000133F6E700ED00E008B572B68A
:101A4000002383F31388FFF7E7FF144B4FF0FF32B7
:101A5000C3F88020C3F88420C3F88820C3F88C2002
:101A6000C3F89020C3F89420C3F89820C3F89C20B2
:101A7000C3F88021C3F88421C3F88821C3F88C21DE
:101A8000C3F89021C3F89421C3F89821C3F89C218E
:101A900062B6BFF34F8FBFF36F8F08BD00E100E068
:101AA000044800232021C2180133302B82F8001390
:101AB000F9D1704700E100E0064B9B68834207D1F3
:101AC000EFF3058323B1044A536843F08053536016
:101AD00001F022BD7808002000ED00E0024B034A2F
:101AE0000348012100F06EB800000420000000202F
:101AF00044490000426E054B203A1A60044A2021F6
:101B0000C3E901121846012100F066B8BC070020A5
:101B100000000B15F0B51F4F00268E4201DB10466A
:101B2000F0BD44689CB353B104F1FF3C14EA0C0FC0
:101B300018D11F2C16D905681CEA050F12D1202CCC
:101B40000568D0F808C0D2B20FD9B4F1004F0ED852
:101B5000013CB4FA84F4C4F11F046400072A4CEA7F
:101B6000040406D96FF01502D9E70824F6E73E24ED
:101B7000F4E725F01F05154345F0100544F0010476
:101B8000C7F89820C7F89C500132C7F8A04001362A
:101B90000C30C2E700ED00E0044B0522C3F89420AE
:101BA000BFF34F8FBFF36F8F704700BF00ED00E0B2
:101BB000BFF35F8F024B0022C3F89420704700BF31
:101BC00000ED00E010B5034C01232278FFF7A2FFDF
:101BD000207010BDD008002008B5094A00231278F3
:101BE000FFF798FF10F1160F02D0064A072800DD14
:101BF00008BDC2F89800C2F8A0300130F6E700BF77
:101C0000D008002000ED00E014490868082810B54D
:101C100021D8FFF7CDFF124C49680022904201F114
:101C20000C0105D10F4B1870FFF7B6FF002010BD57
:101C3000C4F8982051F80C3C23F01F03134343F0E1
:101C40001003C4F89C3051F8043C43F00103C4F87D
:101C5000A0300132E2E74FF0FF30E8E750490000E2
:101C600000ED00E0D0080020014B1860704700BF75
:101C7000280000204FF02003EFF3118283F3118836
:101C8000BFF36F8F06490123C1F840354FF0804103
:101C9000C1F8783582F31188BFF36F8F0020704749
:101CA00000E001404FF08043C0B2C3F81C05BFF311
:101CB0004F8F0549054BCA6802F4E0621343CB60BD
:101CC000BFF34F8F00BFFDE700ED00E00400FA0511
:101CD00020B1034B800143F001031847704700BF58
:101CE000E04800002DE9F0411A4D002701266C79EB
:101CF000D5F80080404602F038FB40B3AB79297933
:101D0000002B14BF4FF4D0534FF4B0532343D8F8F3
:101D10001040D8F808E02068DA0748BF83F4406331
:101D200023F4805206FA01FCDB074CBF4CEA0000AA
:101D300020EA0C002060DEF800304046984720B9C9
:101D400001370F2F05F10805D1D1BDE8F0816FF003
:101D50001200FAE77049000008B5094B1A786AB911
:101D60000121197006200521FFF774FC0620FFF7FA
:101D700053FC044B4FF00042C3F80423002008BD7D
:101D8000D1080020006000402B4BF0B544682B4880
:101D90001340834241D00DD8062B15D005D89BB1F6
:101DA000022B3CD06FF0150036E0B3F5801FF9D15F
:101DB000012309E02248834233D0B3F5A00F32D08B
:101DC000B3F5800FEED10223D00654BFC2F3401604
:101DD000032682F480759705C2F34020C5F30025E1
:101DE00007D512F4006F67681FD001228A40C7F838
:101DF0000825227A134C012A01F01F0140EA45020E
:101E000018BF4FF0A04442EA032301F5E07143EA12
:101E1000860344F821300020F0BD0723D4E70423D3
:101E2000D2E70523D0E70323CEE7520542BF0122C4
:101E30008A40C7F80C25DCE70600F0000600100019
:101E4000020040000003005000F01F024009084B50
:101E5000012818BF4FF0A04303EB8203D3F80027FB
:101E600022F4403242EA0142C3F80027704700BF23
:101E7000000300502DE9F84F0369D0F804A0DE6894
:101E8000DFF87CB08846D3E905210A4326EA02063A
:101E9000DAF804201B69D2F810555D4026EA0505E2
:101EA000374601244FF0000917B92846BDE8F88FDE
:101EB0003C4221D09AF8083009F01F00344240EA31
:101EC000431014D14209012A00F01F0314BF4FF040
:101ED000A0425A4603F5E07352F82330C3F301439E
:101EE000022B02BFD8F800302343C8F8003000218D
:101EF000FFF7AAFF27EA040709F101096400D3E705
:101F000000030050F0B5002485B0CDE90044CDE9D0
:101F10000244284ED6F87C516DB102A92648FFF73D
:101F2000A9FF03A900902548FFF7A4FF0190C6F878
:101F30007C41D6F87C3122491E4C00220126944671
:101F4000D4F8043306FA02F0184216D00B68A3B195
:101F500002F5A27304AF54F82330C1F800C0C3F3F4
:101F6000403007EB8000C3F3042350F8107C06FADE
:101F700003F33B4340F8103C0B680132082A01F19F
:101F80000401DDD1009A22B10E4B0B49586802F0D2
:101F9000F7F8019A22B10C4B0849586802F0F0F8A2
:101FA0002DB1054802F0FDF8044802F0FAF805B03A
:101FB000F0BD00BF00600040FC4600001447000078
:101FC00000610040D0070020EC070020F7B5144660
:101FD00042680769127A01F01F05B4F5A03F0E466A
:101FE00045EA421510D16909012905F01F0261492E
:101FF00002F5E07218BF4FF0A04151F82220D0073F
:1020000007D56FF085009AE0B4F5005FF96800F03D
:102010009880FA680121B14011437A69F960012181
:10202000B140B4F5A03F0CBF0A438A437A61BA6954
:10203000B3F5C02F0CBF0A438A43BA613A69B3F5BE
:10204000802F0CBF114322EA01014B4A3961D2F8BB
:1020500004330020DBB200F5A27152F82110C1F365
:1020600005218D4272D123FA00F1C9076ED5830094
:1020700003F1804303F5C043D3F8101521F00101AB
:10208000C3F8101501238340C2F80833C0B200F032
:10209000D5FB28460021FFF7D7FEF868F04010F086
:1020A00001004CD07869F04010F0010455D0BB69B4
:1020B000F340DB075FBF396921FA06F606F0010637
:1020C000C6F102060DF1070054BFF6B2032600F078
:1020D000D5FB2A4B98423DD19DF80720930003F190
:1020E000804303F5C0432D02D3F8101521F44F317E
:1020F00021F44071C3F81015D3F8101505F47C5580
:102100000D4345EA0646C3F81065930003F180438A
:1021100003F5C243002018609DF807101B688B0070
:1021200003F1804303F5C043D3F8102542F00102C8
:10213000C3F81025104A01238B40C2F8043303B0C2
:10214000F0BD0122B24021EA020166E70130082811
:1021500081D19EE76FF01200F1E73969F14001F09B
:102160000101C1F103012846C9B2FFF76DFE204607
:10217000E5E700BF00030050006000400000AD0B29
:10218000036803F01F025B09012B0260024818BFBD
:102190004FF0A040704700BF00030050F0B54B79EE
:1021A000012B2AD0032B25D110268B79032B21D18B
:1021B000CC792CB1012C1DD143685B689B0719D0E9
:1021C0000A7912B1022A15D10E220B684568B3F5BF
:1021D000164F2D6865D02DD8B3F5165F64D016D88C
:1021E000B3F5966F62D00AD8B3F5967F61D0B3F598
:1021F000167F61D06FF0850052E00026D5E7B3F579
:10220000166F5CD0B3F5965FF4D1374B3CE0B3F575
:10221000E14F57D007D8B3F5615F55D0B3F5964F6E
:10222000E8D1324B30E047F61227BB42E2D14FF4FF
:10223000000329E0B3F5613F48D013D8B3F5963FCA
:1022400047D009D84DF6C027BB4244D0B3F5614F03
:10225000D0D14FF46B0317E0B3F5E13FCAD14FF093
:10226000EB7311E0B3F5612F38D008D8204FBB4293
:1022700037D0B3F5E12FBDD14FF0E86304E01D4F37
:10228000BB42B7D14FF08053C5F82435036903C969
:10229000344322430433C5F86C2583E8030000204F
:1022A000F0BD4FF41D03EFE7134BEDE74FF49E2312
:1022B000EAE74FF4A033E7E74FF41C33E4E74FF4C9
:1022C0001D23E1E70D4BDFE70D4BDDE74FF06C73AE
:1022D000DAE70C4BD8E74FF46503D5E74FF07063AE
:1022E000D2E74FF08063CFE700B0130000A04E00AC
:1022F00090D0030040420F000050270000C075003E
:1023000000F03A0000903A01F8B5066905460F461C
:1023100002F094F810B92C4B1B7883B94FF02003CE
:10232000EFF3118483F31188BFF36F8F686801F0B6
:1023300080FF28BB84F31188BFF36F8FEEE764241E
:10234000686801F076FF70B9012001F0D5FF013C0B
:10235000F6D10021212001F0BFF8F0E784F31188C5
:10236000BFF36F8FF5E74FF02003EFF3118483F392
:102370001188BFF36F8F686801F05BFF0028EDD014
:1023800006F8107F69680B680122C3F84465C3F83A
:1023900048250022C3F82021D3F82001C3F8582192
:1023A000D3F858214A68D20641BF0822C3F8002555
:1023B0004FF48002C3F8042301229A6084F3118849
:1023C000BFF36F8FF8BD00BFD20800202DE9F7439F
:1023D0000022054601210220FFF73CF90220FFF709
:1023E0001BF96B682E691C680023C4F800354FF098
:1023F0000509356001A8CDF80490FFF7C1FE019BE7
:102400004FF0010808FA03F3C0F8083501A8CDF829
:102410000490FFF7B5FE019B03F5E073032140F83C
:10242000231001A80191FFF7ABFE019B03F5E073B8
:102430000C2740F82370C4F80C9501A8C4F81415B3
:102440004FF00709CDF80490FFF79AFE019B03F5C2
:10245000E07340F82370282701A80197FFF790FE4A
:10246000019B08FA03F3C0F8083501A80197FFF7AC
:1024700087FE019B03F5E07340F823102969C4F837
:1024800008750431C4F810952846FFF787FE074603
:10249000002844D16B685B68190719D506F1120052
:1024A00000F024FA214B98423DD1B07CC30003F1E7
:1024B000804303F5F83304F10C0204F59071C3F87E
:1024C0001015C3F814251A4A08FA00F0C2F80405DA
:1024D0000823C4F800350023C4F81031D4F81031B3
:1024E00006F11103C4F834350123C4F838352360EC
:1024F0006B685B681A075CBF4FF48072C4F80423F2
:10250000DB0644BF4FF48003C4F8043310360023C5
:10251000C4F84465C4F848350123A360E360384635
:1025200003B0BDE8F0836FF00407F8E70000AD0BDF
:1025300000F001404FF08053D3F83021082A06D133
:10254000D3F83431052B02D8024AD05C7047002002
:10255000704700BF9C4B0000024AD2F80034002BA9
:10256000FBD0704700E0014010B501F0BBFE40B168
:102570004FF080430022C3F80C21C3F81021C3F8A8
:10258000382501F0AFFE002846D04FF08052604B56
:10259000D2F80414C3F82015D2F80814C3F824158F
:1025A000D2F80C14C3F82815D2F81014C3F82C155F
:1025B000D2F81414C3F83015D2F81814C3F834152F
:1025C000D2F81C14C3F84015D2F82014C3F84415EF
:1025D000D2F82414C3F84815D2F82814C3F84C15BF
:1025E000D2F82C14C3F85015D2F83014C3F854158F
:1025F000D2F83414C3F86015D2F83814C3F864154F
:10260000D2F83C14C3F86815D2F84014C3F86C151E
:10261000D2F84424C3F87025FFF78CFF18B13D4B66
:102620003D4AC3F88C26FFF785FF18B13B4BFB22D0
:10263000C3F81825FFF77EFF70B14FF080414FF0CF
:102640008053D1F8E42ED3F8583222F00F0203F071
:102650000F031343C1F8E43EFFF76CFF20B1304B8A
:102660004FF40072C3F8402601F03CFE48B14FF031
:102670008043D3F80024D20744BF6FF00102C3F8AF
:1026800000244FF08053D3F83021082A0ED1D3F81C
:102690003431052B02D8234AD35C3BB14FF01023D1
:1026A000D3F808224FF08043C3F858254FF0102389
:1026B000D3F80022002A03DBD3F80432002B22DAFD
:1026C000194901234FF01020C1F804351224FFF7F7
:1026D00043FFC0F80042FFF73FFFC0F80442FFF796
:1026E0003BFF0023C1F80435FFF736FFBFF34F8FE0
:1026F0000E490F4BCA6802F4E0621343CB60BFF38C
:102700004F8F00BFFDE70B4B0B4A1A6010BD00BF97
:1027100000C00040005000404881030000F000402D
:1027200000900240964B000000E0014000ED00E008
:102730000400FA05400000200090D003044B1A79F1
:1027400022B9012218609A800248704702487047F7
:102750000C0800200000AD0B0C00AD0B38B510B11B
:10276000012817D038BD4FF080440223C4F8083345
:10277000C4F80401D4F804310123E36042F2107577
:10278000D4F81834DB03EDD5012001F0B5FD013D8F
:10279000F6D1E7E74FF080440023C4F80803C4F8FB
:1027A0000031D4F80031606042F21075D4F80C3476
:1027B000D4F80C24D20303F0010305D523B1012082
:1027C00001F09AFD013DF1D1014B00225A71C9E798
:1027D0000C0800204FF0804310B5D3F800216AB1F7
:1027E0000022C3F80021D3F800210122C3F80823F6
:1027F000114B587910B95A711B6898474FF08043B4
:10280000D3F8042172B10022C3F80421D3F80421C3
:10281000D3F81824D3F81814920704D10122C3F86E
:1028200018259A6010BD0222C3F80823024BBDE8A8
:1028300010401B68012018470C080020012303FAF0
:1028400000F0C3B293B14FF02003EFF3118183F393
:102850001188BFF36F8F064AD36D23EA0000D0655D
:1028600081F31188BFF36F8F0248704702487047A9
:10287000140800200000AD0B0400AD0B2DE9F04161
:102880000546DFF85CE01748DFF85C800024FF2293
:102890000126E3B24FF02001EFF3118C81F3118890
:1028A000BFF36F8F22FA03F1C9070AD5DEF85C1077
:1028B00006FA03F7394201BF3943CEF85C104046AF
:1028C0002B708CF31188BFF36F8F404505D006FA4B
:1028D00003F39A4304F10104DBD1BDE8F08100BFAA
:1028E000140800200200AD0B0000AD0B2DE9F041F3
:1028F000144A154E154F0546154800244FF0010E99
:102900005FFA84FC4FF02003EFF3118883F3118802
:10291000BFF36F8F0EFA0CF3134207D031680B42EE
:1029200001BF1943316085F800C0384688F311882B
:10293000BFF36F8FB84203D09A4304F10104DFD193
:10294000BDE8F081FFFF0F00740800200000AD0B10
:102950000200AD0B0E4B70B553F82040013053F818
:102960002060A64200D870BDD4E9003528469847BB
:1029700065B1EB6830B10028B8BF4042FF28A8BF5E
:10298000FF2018705A7842F001025A700834E8E7C4
:10299000404A000070B5054610B90024204670BDBD
:1029A0000378002BF9D00E4C0E4EB44208D10C4CDB
:1029B000B442F2D0204601F0D8FC50B91834F7E701
:1029C000204601F0D2FC10B12368AB42E6D01834A7
:1029D000EBE72168284601F036FB0028EED1DDE761
:1029E000B44600002C4700000248034A0021121A96
:1029F00001F040BB00010020900A002008B50A4BFE
:102A0000012202201A70FFF7A5FF00F02BFF032020
:102A1000FFF7A0FF00F016F901F011F9034A137B4C
:102A200023F00103137308BDD208002080010020A9
:102A30002DE98048DFF8E090A7B089F30888374D8A
:102A4000374E6B69DFF8DCA0374F43F40073002486
:102A50006B61E02385F82230EC772C766C76AC76CF
:102A60006B6A43F4E0236B62FEF7C0FFFEF752FE91
:102A70004FF0FF33AB62EB62FFF7C6F82B4DFFF769
:102A80002DF840F20113ADF8243006ABAB60CDE970
:102A90001F4401F069FC2046FFF75CFF0120FFF7AF
:102AA00059FF4FF0010B00F083FC214B6E6221496E
:102AB00005934FF480625346CDE9034BCDE90144C1
:102AC0000094304600F08CF8737B804623F00403BA
:102AD0003046737301F026FD0F23CDE902431649FA
:102AE000164B4FF4A072CDE904B4CDE9005438463A
:102AF00000F076F87B7BEF6023F004037B7305F135
:102B00001803C5E906332C75C5F8049052464146B2
:102B10003046FEF7E9FD00BF4018002000ED00E060
:102B200080010020FD29000000010020780800201D
:102B3000A24B0000A00A0020C00E0020FD2C0000C7
:102B400070B50E4B0E4CA34201D3002070BDD3E9EB
:102B5000030141EA000212F003020BD19D685A61A1
:102B6000AA4201D11C33EEE75E690E600132596161
:102B70000144F5E76FF01500E8E700BFAC00002066
:102B8000AC00002037B50C464FF02005EFF3118163
:102B900085F31188BFF36F8F45695DB125602B68A0
:102BA0004361836901338361002081F31188BFF39E
:102BB0006F8F11E052EA030C03D125606FF00B0018
:102BC000F3E7CDE900230246083000F079FA18B99E
:102BD000024B9B685B69236003B030BD780800201E
:102BE0002DE9FF410E9E0673042646730D9E8673E3
:102BF00000F158050F46D61DC0E916550C9A002560
:102C000026F007062037C0E90655C0E91976856029
:102C1000C573C56606F1200802920B9A019288449A
:102C20000A9A009242460446FEF72CFD044B656565
:102C30009B6803B11B6F2367404604B0BDE8F08179
:102C4000780800202DE9F043294C2A4D87B026460C
:102C5000AE4204F130040FD300F0C0F9244CDFF889
:102C600098904FF4004640F2E737AC4220D307B0CB
:102C7000BDE8F04300F06ABA54F8043C059354F8F8
:102C8000103C049354F8143C039354F8183C0293FA
:102C900054F81C3C019354F8203C009354E90C0177
:102CA00054E90A23FFF79CFF54F8303C5E65CEE7F9
:102CB000636A5A1C0DD023EAE37300213846C3FB34
:102CC000060151EAC333D4F8008004D1404600F035
:102CD00009FB3034C9E74FF47A720023FDF710FA8C
:102CE00002460B4608F11800494600F0CDFCF0E71B
:102CF000AC000020AC0000204545000008B5094CA0
:102D00004FF02002EFF3118382F31188BFF36F8F2E
:102D100001F068FC2062FEF793F80028F0D1FEF77E
:102D2000FFFCEDE7780800202DE9F3410446174643
:102D30001E464FF02003EFF3118883F31188BFF391
:102D40006F8FC368324A6BB180689168884219D02E
:102D500057EA060318D188F31188BFF36F8F6FF01D
:102D60000F000CE0916891F90E1021610133E360CE
:102D70009368A36088F31188BFF36F8F002002B0BF
:102D8000BDE8F0812169F0E791F90E1090F90E305D
:102D90009942A8BF19466FF07E029142B8BF114612
:102DA0008B422EDD01F057FB0546CDE90076194830
:102DB0002246414600F084F90028E0D04FF020037D
:102DC000EFF3118683F31188BFF36F8F23682169B6
:102DD0009C420AD04BB193F90E309942A8BF1946D4
:102DE0006FF07E039942B8BF1946A06801F033FB2B
:102DF00000B945B10748314600F0DEF86FF00A002F
:102E0000BDE70025D1E786F31188BFF36F8FF5E7A3
:102E100078080020D308002038B583680446002BCA
:102E200032D01C4A9268934231D1DA7B013ADA738C
:102E3000C368012B05D9013BC36000F087F900206E
:102E400038BD4FF02003EFF3118583F31188BFF3F2
:102E50006F8F0169806801F0FEFA204601F094FB53
:102E6000A06058B190F90E2022610022826701F023
:102E700059FB0948294600F09FF8DEE7E06085F33A
:102E80001188BFF36F8FD8E76FF01500D8E74FF0C8
:102E9000FF30D5E778080020D308002038B5044675
:102EA0004FF02003EFF3118583F31188BFF36F8F89
:102EB00001F06AFB48B10022826701F033FB29462A
:102EC0000548BDE8384000F077B8D4E902329A42AC
:102ED00018BF0133A360F2E7D308002013B54FF009
:102EE0002004EFF3118184F31188BFF36F8F84689E
:102EF00044B1013C846081F31188BFF36F8F0020DF
:102F000002B010BD52EA030406D181F31188BFF369
:102F10006F8F6FF00F00F3E7CDE900230246024800
:102F200000F0CEF8ECE700BFD308002010B5084C45
:102F300023685BB1FEF744FA03462068054A034460
:102F4000BDE810401361002101F05CBB10BD00BF63
:102F5000B008002078080020F8B504460D464FF070
:102F60002003EFF3118683F31188BFF36F8F0F4BAC
:102F700000214FF4004740F2E73019614FF47A72B4
:102F80000023E4FB0701FDF7BBF8002C084B09DC2C
:102F90001860084B1D60FFF7C9FF86F31188BFF367
:102FA0006F8FF8BD0228B8BF0220F1E77808002033
:102FB000B0080020AC08002049B9EFF3058030B913
:102FC000054B5A6A9B689A4201D0FEF7D1BA81F349
:102FD0001188BFF36F8F7047780800204FF02003EF
:102FE000EFF3118183F31188BFF36F8F044B9A685D
:102FF000D37B013BD37381F31188BFF36F8F70478D
:103000007808002038B502460C480D4D01F05AFAF8
:10301000044600B9EC68AB684AB95A7BD20606D1BF
:10302000A26922B9DA897F2A01D96B6238BD9C4234
:1030300001D0FFF77BFF6C62F8E700BFA00800201B
:103040007808002008B590F90D20437B002A01463E
:1030500004DA03F07F03437301F00CFA044B986821
:10306000431A58425841BDE80840FFF7CBBF00BFA4
:10307000780800202DE9F041064615461C464FF021
:103080002003EFF3118783F31188BFF36F8F01F0F3
:103090001FFA87F31188BFF36F8FB4F1FF3F08BFAA
:1030A000B5F1FF3F08D02A46234606F11800034930
:1030B000BDE8F04100F0E8BABDE8F0814545000008
:1030C00010B5074B9868074B0C4618601146DDE9B0
:1030D0000223FFF7CFFF2046BDE81040FEF748BAB5
:1030E00078080020A808002070B50446183001F0C8
:1030F00063FA4FF02003EFF3118683F31188BFF3D7
:103100006F8F94F90D20637B002A05DA03F07F03AB
:103110006373204601F0AEF90B4D637BA86843F062
:1031200010036373031B58425841FFF76BFF86F38C
:103130001188BFF36F8FAB68A34203D1BDE8704025
:1031400001F0B6B970BD00BF7808002010B54FF08F
:103150002003EFF3118483F31188BFF36F8F084BC3
:103160009A68D37B0133D3730020FFF74BFF84F3BE
:103170001188BFF36F8FBDE8104001F099B900BF0F
:103180007808002070B590F90D20437B002A014695
:1031900004DA03F07F03437301F06CF94B7B154AAB
:1031A00063F07F034B73D2E90A3402F12805AB4286
:1031B0001BD0D3B191F90E6093F90E0086420FD067
:1031C000801B00280CDD5868C1E90030016059609F
:1031D0009068431A5842BDE870405841FFF712BF4B
:1031E000A34202D01B68002BE6D1C1E90054216044
:1031F000D162EDE77808002038B501464FF0200392
:10320000EFF3118483F31188BFF36F8F154B164AC8
:1032100098681568A84206D1FFF788FE84F31188E4
:10322000BFF36F8F38BD00251560104A1268BAB120
:10323000C2897F2A14D8427BD20611D10C4A90F958
:103240000E50126895420BDB0A4A904208D01A6968
:103250008A4202DCFFF796FFDEE7521A1A61DDE7C9
:103260000022FBE778080020A8080020B008002012
:10327000AC0800200001002070B490F90D20437BC1
:10328000002A2ADBDA0628D1826932BB144A63F0AD
:103290007F034373D2E90A3402F12805AB4217D009
:1032A000B3B190F90E6093F90E108E420BD0891BCA
:1032B000002908DD5A68C0E900321060586070BC0F
:1032C0000020FFF79FBEA34202D01B68002BEAD16B
:1032D000C0E900542060D062F1E770BC704700BFC5
:1032E0007808002010B54FF02002EFF3118482F32C
:1032F0001188BFF36F8F427B510704D484F3118888
:10330000BFF36F8F10BD22F004024273FFF7B4FFCA
:1033100021460248BDE81040FFF74EBED30800200A
:10332000F8B504464FF02003EFF3118683F31188BC
:10333000BFF36F8F437BDA0649B233D182698ABB10
:1033400003F07F03437301F095F8437B174A8173C1
:1033500063F07F034373104650F8283F83421BD02D
:10336000D3B1D76A93F90E50A94210D06D1A002D2F
:103370000DDD5A68C4E9003214605C600120FFF77B
:1033800041FE012086F31188BFF36F8FF8BDBB4269
:1033900002D01B68002BE5D1D36AC4E900031C608E
:1033A000D462EBE7A1730020ECE700BF78080020AF
:1033B000044B002103F12802C3E90A220846FFF763
:1033C000CBBD00BF78080020F8B54FF02003EFF325
:1033D000118583F31188BFF36F8F1A498868437B87
:1033E00003F07F03437301F045F88B685A7B08466E
:1033F00062F07F025A7350F8282F82421CD0DAB153
:10340000CF6A93F90E6092F90E40A6420FD0A41B2A
:10341000002C0CDD5168C3E900210B6053600120D2
:10342000FFF7F0FD2846BDE8F840FEF7A1B8BA4224
:1034300002D01268002AE6D1CA6AC3E9000213600A
:10344000CB62ECE77808002050EA01032DE9F04157
:1034500005460E4603D1FFF7B7FF002033E06FF0BB
:103460000104241A4FF0FF3363EB0103012C73F1C5
:10347000000302DA01F0E0F844194FF02003EFF303
:10348000118883F31188BFF36F8F104F104BB8680A
:103490001860FFF7D7FDB8680E492A463346183042
:1034A00000F0F2F8BA68537B43F0100353734046C0
:1034B000FEF75EF801F0C0F8201A63EB0303012861
:1034C00073F10003C9DBBDE8F08100BF780800207C
:1034D000A808002045450000B1F1FF3F08BFB0F14A
:1034E000FF3F08B506D1084B9868FFF7FDFD4FF088
:1034F000FF3008BDFFF7A8FF4FF47A7380FB03038A
:10350000C00B40EA4340F4E778080020014B98687C
:10351000704700BF780800202DE9F04104464FF0C5
:103520002003EFF3118683F31188BFF36F8F437B82
:103530001A0705D586F31188BFF36F8FBDE8F081B8
:1035400023F0200242F00801D20920D14173A36880
:1035500013B1204600F096FF04F1180001F02CF89A
:1035600004F158074FF00008A56DBD4200D0B5B971
:103570000120FFF747FD104B9B68A342DAD1EFF320
:103580000583002BD6D13046FDF7F2FFD2E703F0DA
:103590005F0343F00803437300F06CFFD7E728464E
:1035A00000F070FF05F1180001F006F8C5F878800A
:1035B0002846FFF761FED7E77808002008B50648DF
:1035C000064A0749121A00F04AFDBDE80840054ABC
:1035D0000549064800F043BD00000020FC00002023
:1035E000E04B000000000000E04B00000000002065
:1035F000034B1B680BB9FDF7E3BE0020704700BF0B
:10360000B4080020114B10B51C689C4208BF002470
:10361000FFF7EEFF03466CB1D4E90402C01A62EB77
:10362000E373012873F100020DDBB0F1004F73F179
:10363000000301DB6FF00040054B1B6913B198429A
:10364000A8BF184610BD0020F6E700BF44000020C8
:103650007808002030B5036868B10A4A5268904281
:1036600009D043B1D3E90421D0E90445121941EB53
:103670000501C3E90421426813605A600023C0E9D0
:10368000003330BD44000020B3F1FF3F08BFB2F16A
:10369000FF3FF8B504461F46154667D081604FF0DE
:1036A0002003EFF3118683F31188BFF36F8F6FF060
:1036B0000102531B4FF0FF3C6CEB0703002B1BDB9D
:1036C0002B4BD3E90013521A6CEB0303551B63EB2E
:1036D0000703012D73F10002BCBF01250023C0E9DF
:1036E00004532448D0E9003C834218D1C4E9000CBB
:1036F000CCF80040446026E0FFF77AFF013547F13F
:1037000000072D1847EBE077C4E90457E9E7521AA0
:1037100065EB07059C45C4E90425E7D01B68002B31
:10372000E4D0D3E90417D4E904258A4275EB070EE7
:10373000EDDA8A1A67EB0505C3E904255A68C4E97E
:10374000003214605C60036883420BD09C4209D154
:10375000FFF758FF18B1084B1B69834202D00021C4
:10376000FDF7FCFD86F31188BFF36F8FF8BD00BF36
:103770000002002044000020780800202DE9F843D2
:103780000546FFF739FD4FF02003EFF3118483F373
:103790001188BFF36F8F244EDFF890803560244D81
:1037A000D8F8000032684045D5E9001E4FEAE277BC
:1037B0000BD050B1D0E9043C9A4277EB0C0916DAF1
:1037C0009B1A6CEB070CC0E9043C52184EEB070740
:1037D000C5E9002700253560FFF714FF2946FDF7EE
:1037E000BDFD84F31188BFF36F8FBDE8F8835918CE
:1037F0004EEBE377D31A336000220023C0E90423A1
:10380000C5E90017FFF726FF84F31188BFF36F8F18
:10381000836898474FF02003EFF3118483F31188F6
:10382000BFF36F8FBCE700BFB40800204400002046
:103830000002002010B54FF02003EFF3118483F352
:103840001188BFF36F8FFDF7BBFD054AD2E9003148
:10385000C01841F1000184F31188BFF36F8F10BDD0
:1038600000020020024A0349034800F00FBA00BFDB
:10387000DC4B0000A74B0000B64B000010B50A4C13
:1038800023681BB101232360002010BD00F0D6F88F
:103890000028F7D00138062803D8044B53F820003D
:1038A00010BD034810BD00BFB8080020584A0000F2
:1038B000FE8FFFFFBFF34F8F0549064BCA6802F426
:1038C000E0621343CB60BFF34F8F00BFFDE700BF43
:1038D00000ED00E00400FA05F0B4094F094E0A4C6F
:1038E0000A4A0B4D0B494FF0FE333B605268336080
:1038F000236000242B60C1F80045F0BC104700BFD6
:1039000000B4025004B4025008B402504C0000202D
:103910000CB4025000A00250D0E90012014BC3E9E0
:10392000001270474C00002010B5044630B16368A7
:10393000DB0602D500232360636010BD024B034801
:103940005B689847F3E700BF4C000020744A000012
:1039500068B143683BB1DB0607D5BFF35F8F002337
:1039600003601846704703487047034870476FF478
:10397000E0407047EA8FFFFFE98FFFFF10B5044674
:1039800020B1002211232260636010BD0148FFF7BF
:10399000A3FFF6E79C4A0000C0B14368A3B1DB0671
:1039A00010D50122BFF35B8F50E8003F40E80021B3
:1039B0000029F9D1BFF35B8F012BF3D0BFF35F8FE9
:1039C0000020704703487047034870476FF4E04099
:1039D000704700BFE98FFFFFEA8FFFFF70B5D0E9A6
:1039E0000023134C134DC4E90023D0E90263C4E95A
:1039F0000263114B086818604868586088689860CE
:103A0000D1E90360D5F81411DE601861CB060DD53D
:103A10000023C5E94433C5E96D3305F58870904747
:103A2000236805F5DA70BDE87040184770BD00BF27
:103A30005C000020D40800206C00002010B500F0CD
:103A400033F820B1032400F067F8204610BD00F0E1
:103A500035F890B900F0B0F890B90F4B1B681B0E09
:103A6000F02B08D10D4A0E4B12689A420AD0072457
:103A700000F01CF8E7E70624FAE70424204610BD0E
:103A80000024F5E7012000F097F804460028F7D15C
:103A9000044B1860D9E700BF28B9025024BA02507D
:103AA0000000E0200CBA0250002070470020704750
:103AB000014B1860704700BF04BA025010B511489E
:103AC00000F048F800B110BD0F4800F043F800289E
:103AD000F9D10E4C204600F03DF80028F3D10C4BF4
:103AE0000C481C6000F036F801460028EBD100F0CD
:103AF0002DF8044608B1204610BD00F03FF82046DE
:103B0000FAE700BFA400002098000020A0000020D9
:103B1000A80000209C00002008B5084800F024F808
:103B2000074800F021F8074800F01EF8064800F0AA
:103B30001BF8BDE8084000F00BB800BFA40000204F
:103B400098000020A00000209C000020002070476A
:103B5000704700BF08B5034B02681B6810689847A0
:103B6000002008BD5C00002008B5034B02685B68BC
:103B700010689847002008BD5C00002070B5094C13
:103B8000094D2069AB68984718B1084B08485B6835
:103B90009847084AEB68206900211160BDE8704031
:103BA000184700BF6C0000205C0000204C00002083
:103BB000C04A0000CC08002070B51A4D1A4E0446C9
:103BC000B26828699047F0B95CB1184C2368ABB172
:103BD000012B1AD0013B23602869F3689847002025
:103BE00070BD124C216839B9114B124A0120C3F83B
:103BF00000051368002BFCD101312160F3682869AE
:103C00009847002070BD0C4870BD0A4A1368002B0D
:103C1000FCD1074A6FF07E40C2F80035FFF748FF3D
:103C20002368D7E76C0000205C000020CC0800204F
:103C300000A0025010B90250E98FFFFF704708B58D
:103C400000214FF40040FFF747FCF9E7034658B165
:103C5000426802F00302012A03D0032A04D1026859
:103C600012B10020986070476FF0150070474268ED
:103C7000816002F00302032A4FF0000203460CBFEA
:103C8000006810465A607047002070470FB407B5AF
:103C900004A951F8040B0191FCF7C2FB03B05DF8D5
:103CA00004EB04B07047038B13F0070305D10368DE
:103CB000002B0CBF002003207047022B05D1438B43
:103CC000002B14BF002004207047012B05D103688E
:103CD000002B0CBF002005207047002070472DE905
:103CE000F0410D4607461946281D90461E46FFF72F
:103CF000BEFF044638B13346424629463846A446FC
:103D0000BDE8F0416047BDE8F08110B44FF02004F9
:103D1000EFF3118284F31188BFF36F8F416110BC00
:103D20000121FCF78BBB10B50C4640B139B1081D21
:103D3000FFF78CFF28B9A36833F0030301D06FF0BD
:103D4000150010BD38B50C46054658B151B10B6889
:103D500043B14B6833B11C22002100F08BF92C6178
:103D6000002038BD6FF01500FBE770B504460E4625
:103D7000FFF7D9FF051E31DB4FF02003EFF3118170
:103D800083F31188BFF36F8F638B208B4FF6FF7522
:103D9000AB4200F007022ED0022A0ED1013363831A
:103DA0001546012381F31188BFF36F8FB3B1002350
:103DB00031462046FFF793FF10E0830701D0062A23
:103DC0000ED100233360636893B9C4E900661546D9
:103DD00062B90A4620460221FCF730FB284670BD36
:103DE000052A0CBF6FF085056FF004050023D9E7A5
:103DF0001E606660EBE76FF00A05F7E7044608B55A
:103E0000084611461A46A047FFF780FBFDF754FE0F
:103E10002DE9F84F9A46D3786F2B80460F4615460A
:103E2000A3F1410B29D024D8582B14BF0A26102601
:103E3000DDF828903246002340463946FCF760F909
:103E4000092AD4B21ED83034B045E4B277F1000369
:103E500009F8014D01D3D14511D82B789B0605D522
:103E6000082E15D1AB7843F00803AB704846BDE887
:103E7000F88F03F0F703702BD7E70826D8E78046C2
:103E80000F46D7E7BBF1190F94BF37345734DBE740
:103E9000102EEBD1AB7843F01003E6E72DE9F041AB
:103EA0000746884615461E461446B442A4EB050054
:103EB00002D33EB923782BB114F8010B4146B84721
:103EC0000028F2DABDE8F08170470022C0E9002244
:103ED000826070470369C9B20C2201FB0233186C7F
:103EE00000F0070070474FF02003EFF3118283F3D7
:103EF0001188BFF36F8F036803F0C00343F0020320
:103F0000036082F31188BFF36F8F7047034670B56B
:103F10000069C9B24FF02004EFF3118684F31188D1
:103F2000BFF36F8F0C2505FB0104246C14F0C00453
:103F300001D0A24210D105FB010001220264002041
:103F400086F31188BFF36F8F28B95B6803EBC1015B
:103F50004B689847002070BD4FF0FF30F0E780229B
:103F6000FFF7D4BFF8B5069F04690546C9B24FF004
:103F70002000EFF3118C80F31188BFF36F8F0C26B4
:103F800006FB0146306C00F0070EBEF1010F11D1A7
:103F9000376400268CF31188BFF36F8F46B90C206D
:103FA00000FB0144C4E90E236B6853F83130984795
:103FB0003046F8BD00F0C000874214BF4FF0FF3616
:103FC0006FF07706E6E713B580240094FFF7CAFF89
:103FD00002B010BD006910B4CBB21C2403FB040076
:103FE000002110BC1047002000F092B90020FEF71D
:103FF000B5BB1046FEF752BF7047704770470020B0
:10400000FCF7BEBE0021012000F000B800F0B7B9F7
:104010000146006800F0B3B908B5FDF799FBBDE8AB
:104020000840FDF7EBBC034600201A5C02B970475C
:104030000130FAE7034600201A5C0AB1884200D139
:1040400070470130F8E7431E013913F8012F11F8CA
:10405000010F824201D1002AF7D1101A704710B522
:10406000431E0A44914200D110BD11F8014B03F8E0
:10407000014FF7E7C9B202440346934200D17047AB
:1040800003F8011BF9E74FF0FF30704784B004AB31
:1040900003E907009DF80430062B08D14FF0804358
:1040A0000122C3F80025BFF34F8F20BFFDE704B006
:1040B000704784B004AB03E90700002383F3118841
:1040C000BFF36F8F04B070474FF0A0434FF400224E
:1040D000C3F808250322C3F84C2700207047436823
:1040E0005B68D3F810350B600020704743685B684D
:1040F000D3F8040542400A404240C3F8042500209A
:10410000704743685B680020C3F808157047436830
:104110005B680020C3F80C15704743685A68D2F8F2
:1041200004354B40C2F804350020704703695868D5
:1041300030B558B10024814212D108689D6854B945
:104140008D42586000D19860002008606AB9002054
:1041500030BD2846EFE78D42206008BF9C60F3E742
:1041600005680446002DF4D13AB198685A680A608F
:1041700059600028EBD19960EAE76FF01500E7E796
:1041800070B50E461546014650B104688A682A404B
:1041900002D04B683046984714B121462468F5E7B1
:1041A00070BD2DE9F0410769D0F80480FC68D7E9BB
:1041B0000532134324EA0304012600250CB9BDE8A7
:1041C000F081264210D0396998F80830E94001F0B2
:1041D0000101C1F1030105F01F00C9B240EA43101B
:1041E000FDF732FE24EA060401357600E6E70269AF
:1041F0000B46D2E9010183E80300002070474368C1
:104200001B68D3F88004C3F88004704743680269D0
:104210001B68D3F8100148B1527C0A700020C3F823
:104220001001D3F8102101221A6070474FF0FF30BF
:10423000704702680346D2F8580140B95B681B0713
:1042400006D4D2F82001003818BF012070470120A1
:10425000704743681B68D3F80423D10518D5D3F8F9
:104260002021AAB14FF02001EFF3118281F31188D0
:10427000BFF36F8FD3F8201131B10021C3F82011A3
:10428000D3F820110121D96082F31188BFF36F8F19
:1042900042685268D20615D54FF02001EFF3118223
:1042A00081F31188BFF36F8FD3F8581111B100213A
:1042B000C3F800154FF48001C3F8081382F3118886
:1042C000BFF36F8F704708B50020FDF7EBFCFFF7D9
:1042D000D5BA08B5FDF782F8FDF734F9BDE8084016
:1042E000FFF7CCBA4FF08053D3F83001A0F10803A8
:1042F000584258417047004700F0A2B908B5002065
:10430000FDF79AF918B9BDE80840FDF785B908BD71
:1043100010B101281DD070474FF08043D3F8182406
:10432000D3F81814C90312D502F00302012A0ED1E2
:10433000C3F818254FF080430022C3F80421D3F8B6
:1043400004210222C3F8042301229A60704700224C
:10435000EEE74FF080430022C3F80021D3F800219C
:10436000C3F8040318607047704738B1C3681888F1
:10437000C0F30800A0F58073584258417047F8B563
:1043800005460E464FF02003EFF3118783F31188A3
:10439000BFF36F8FFFF7BAF8314604462846FFF7A0
:1043A00092FF87F31188BFF36F8F2046BDE8F84076
:1043B000FDF782BB30B50024846141EA020414F0A9
:1043C0000304C0E9023201610CD14461A34203D16C
:1043D000C0E90000002030BD45690D600134416135
:1043E0001144F3E76FF01500F5E7F8B504460D4604
:1043F0004FF02003EFF3118683F31188BFF36F8F23
:10440000476977B900F0C0F858B12A6842618767F8
:1044100000F088F8314604F10800BDE8F840FEF7E6
:10442000CBBD2B6862691A602B686361A369013B8D
:10443000A36186F31188BFF36F8FF8BDEFF305809A
:10444000003818BF0120704708B5FCF7D3FCBDE861
:104450000840FFF7D2BD90F90E308B4201D0FEF735
:104460005FBF0020704703460020C3E90200C3E994
:1044700000337047D0E9003213605A600023C0E96E
:104480000033704708B5FFF7F5FF437B23F00203C5
:1044900043730023836008BD034620B9EFF3058210
:1044A0000AB9FDF765B883F31188BFF36F8F7047C2
:1044B0004FF02003EFF3118083F31188BFF36F8F68
:1044C000FFF7EABF03460068834208BF0020704739
:1044D00038B504460D46FEF7B5FD637B43F0020395
:1044E000637395B12B68A5609D4215D0A3B194F973
:1044F0000E1093F90E20914208D0521A002A05DDC1
:104500005A68C4E9003214605C6038BD6A6893423E
:1045100002D01B68002BECD16B68C4E900531C600F
:104520006C60F2E710B54FF02003EFF3118483F3D2
:104530001188BFF36F8FFEF79FFE84F31188BFF3DE
:104540006F8F10BD10B501464FF02003EFF31184BB
:1045500083F31188BFF36F8F10F80B3C13F0280F13
:104560000DD151F8103C18380BB1FFF78BFF11F843
:104570000B3C23F0140301F80B3CFEF77DFE84F3A3
:104580001188BFF36F8F10BD38B54FF02003EFF3E4
:10459000118583F31188BFF36F8FFFF793FF0446F4
:1045A00020B1FFF76FFF183000F006F885F311888F
:1045B000BFF36F8F204638BD10B54FF02002EFF3E8
:1045C000118482F31188BFF36F8F03683BB1FFF74B
:1045D00041F8002084F31188BFF36F8F10BD6FF096
:1045E0001500F7E710B54FF02003EFF3118483F3C4
:1045F0001188BFF36F8FFFF705F884F31188BFF3BD
:104600006F8F10BD70B504460D464FF02003EFF3D9
:10461000118683F31188BFF36F8FFEF7F3FF012834
:1046200005DDA04203DB29462046FCF797FE86F312
:104630001188BFF36F8F70BD08B5FFF7FBF808BD99
:0C46400008B1FDF745BB7047FDF78EBFC9
:08464C00E4BAFF7F0100000049
:10465400751C000000000000C940000000000000BC
:10466400412B000000000000CF42000000000000C9
:10467400910F0000B4460000CD230000CC4600009A
:10468400C90E00000000000011130000E446000001
:10469400591D000014470000591D0000FC4600008D
:1046A400D342000000000000E51C000000000000F0
:1046B400164B0000FC480000E848000020020020DF
:1046C40034020020CC4800000F4B0000384A0000A0
:1046D400244A0000080800202C000020C2480000E2
:1046E4001C4B000000000000000000008C020020B1
:1046F40000000000BC4800008F4B00000C4A000082
:10470400E8490000C8070020D0070020B448000092
:10471400884B0000184A0000E8490000CC0700203C
:08472400EC070020AC48000086
:10472C00D5270000F7420000000000000540000003
:10473C00CC46000053420000000000000540000081
:10474C0000000000054000000000000005400000D3
:10475C0000000000051F00000000000005400000E4
:10476C0000000000054000000000000005400000B3
:10477C0000000000054000000000000005400000A3
:10478C000000000005400000000000000540000093
:10479C000000000005400000000000000540000083
:1047AC00000000000540000000000000B1120000F5
:1047BC000000000005400000000000000540000063
:1047CC000000000005400000000000000540000053
:1047DC000000000005400000000000000540000043
:1047EC000000000005400000000000000540000033
:1047FC000000000005400000000000000540000023
:10480C000000000005400000000000000540000012
:10481C000000000005400000000000000540000002
:10482C0000000000054000000000000005400000F2
:10483C0000000000054000000000000005400000E2
:10484C0000000000054000000000000005400000D2
:10485C0000000000054000000000000005400000C2
:10486C0000000000054000000000000005400000B2
:10487C0000000000054000000000000005400000A2
:10488C000000000005400000000000000540000092
:10489C000000000005400000000000000540000082
:1048AC00FF7FFF7FFF7FFF7FFF7FFF7FFF7FFF7F0C
:1048BC00FF7FFF7FFF7FFF7FFF7FFF7FFF7FFF7FFC
:0A48CC00FF7FFF7FFF7FFF7FFF7F6C
:0A48D600FFFFFFFFFFFFFFFFFFFFE2
:1048E0000338FDD870470000A51000005F3F0000AE
:1048F000C73F000000000000D53E0000411000004E
:10490000D9100000E73F0000ED3F00004D0F000010
:104910001D0F00000000000000000000FF3F00002D
:10492000D5140000E91300003114000089140000C0
:1049300020000020080000201800002000000000D7
:1049400010000020000000200000000000000B0606
:10495000020000005849000000000000794B0000F0
:104960002600020700000020814B000022000B11EE
:10497000144700000E010100FC4600000C0001007D
:10498000144700000C00010014470000050101005D
:104990001447000007010100144700000101010055
:1049A0001447000003010100144700000901010041
:1049B000FC46000008010100FC4600000601010061
:1049C000FC4600001A010100FC4600000D0000003A
:1049D000FC46000018000000144700000A00000018
:1049E000FC46000013000100891D0000DF400000AC
:1049F000ED400000034100000F4100001B4100009A
:104A0000CD1F00002D41000000000000FFFFFFFF50
:104A10000000005000000000FFFF000000030050F5
:104A2000010000000D42000009230000FF410000CA
:104A30009D210000EF410000002000400B0000001D
:104A4000544600008C46000094460000B446000026
:104A5000B4460000F5FFFFFFFF8FFFFFFF8FFFFF52
:104A6000FE8FFFFFFE8FFFFFFD8FFFFFFC8FFFFF1D
:104A7000FC8FFFFF6D757465785F667265652063F6
:104A8000616C6C65642077697468204E554C4C20CD
:104A9000706172616D6574657200000043616E271C
:104AA0007420696E697469616C697A65206D7574CA
:104AB00065782C20776173204E554C4C0D0A000010
:104AC000436F756C64206E6F74206C6F636B207025
:104AD0006F7765722073617665206D7574657800F7
:104AE000286E696C29004661696C656420746F20CA
:104AF0007265626F6F743A207370696E6E696E676B
:104B000020656E646C6573736C792E2E2E0A0055C9
:104B10004152545F3000434C4F434B007379735FF5
:104B2000636C6F636B006D757465785F696E697433
:104B30002063616C6C65642077697468204E554C05
:104B40004C20706172616D6574657200436F756CA5
:104B500064206E6F7420616C6C6F63617465206D8E
:104B600075746578206265666F726520696E697418
:104B700069616C697A696E6700464C4153485F30E1
:104B8000005352414D5F30004750494F5F3100475D
:104B900050494F5F3000000000000101010000009B
:104BA00000006D61696E0076322E362E39392D6E19
:104BB0006373312D31002A2A2A20426F6F74696E87
:104BC00067205A6570687972204F53206275696C4E
:104BD00064202573202573202A2A2A0A0000000059
:104BE000893C000001000000AC0000200100000032
:104BF000C000002001000000D400002001000000DF
:104C0000E8000020010000008740000000000000D4
:104C100000C20100000103000000000000000000CD
:104C20000090D00344000020440000200000000059
:104C3000B5380000BC080020110000007D390000DC
:104C400029390000993900005139000090000020F6
:104C50005400002088000020000000008000002098
:104C6000C008002011000000C4080020110000004E
:104C7000C808002011000000700000207C00002007
:0C4C8000740000206C000020A000002048
:104C8C00AC000020AC000020000000000000000080
:104C9C000E000000C0000020C0000020000000003A
:104CAC00000000000E000000D4000020D400002002
:104CBC0000000000000000000E000000E8000020D2
:104CCC00E800002000000000000000000E000000C2
:04000003000017D111
:00000001FF
